:020000040000FA
:1000000008EF10F012001200C3EF01F0120001001F
:100010002C20000060000000400000000F0E93162E
:1000200081160ED9939493968194819609D90F0ED7
:100030008114816E300E8110816E2BD801D90F0E84
:100040008116300E811225D8FBD80F0E8116300E86
:10005000811246D91ED819D90F0E811641D9818A2D
:100060003FD917D8280EE66E19D8E552080EE66E6D
:1000700015D8E552010EE66E11D8E552060EE66E71
:100080000DD8E5520C0EE66E09D8E55229D900D0FC
:100090001200818625D981966AEF01F0D9CFE6FF5B
:1000A000E1CFD9FF1DD9819481960F0E8116FE0EE6
:1000B000DB50F00B811214D9ECDF0F0E8116FE0E0F
:1000C000DB38F00BF00B81120BD9E3DF00D0E552E7
:1000D000E7CFD9FF1200D9CFE6FFE1CFD9FF00D992
:1000E000818481960F0E8116FE0EDB50F00B81127B
:1000F0008186F6D881960F0E8116FE0EDB38F00B46
:10010000F00B81128186ECD8819600D0E552E7CFC2
:10011000D9FF1200D9CFE6FFE1CFD9FFFD0EDBCF2B
:10012000F6FFFE0EDBCFF7FF0800F55011E0FD0EE5
:10013000DBCFF6FFFE0EDBCFF7FF0800F550E66ED3
:10014000CADFE552FD0EDB2AFE0E01E3DB2AE6D70D
:1001500000D0E552E7CFD9FF1200D9CFE6FFE1CFBB
:10016000D9FFFD0EDBCFE9FFFE0EDBCFEAFFEF503C
:1001700010E0FD0EDBCFE9FFFE0EDBCFEAFFEF5014
:10018000E66EA9DFE552FD0EDB2AFE0E01E3DB2A57
:10019000E8D700D0E552E7CFD9FF1200D9CFE6FF6C
:1001A000E1CFD9FFE652FE0EDB0404E1FD0EDB5089
:1001B000800FDF6EFE0EDB50020804E1FD0EDB5007
:1001C000C00FDF6EDFCFE6FF69DFE552E552E55293
:1001D000E7CFD9FF1200D9CFE6FFE1CFD9FF020E5A
:1001E000E126E66AFE0EDBCFE6FFD8DFE552E552F8
:1001F000DE6ADD6ADECF14F0DDCF15F0D890155041
:1002000004E6100E145C000E155809E2200EE66E8E
:1002100062DFE552DF2A010E01E3DB2AEBD7E66A53
:10022000FE0EDBCFE6FFBADFE552E552020EE15CDF
:1002300002E2E16AE552E16EE552E7CFD9FF120032
:10024000D9CFE6FFE1CFD9FF020EE126DE6ADD6AF3
:10025000DECF14F0DDCF15F0D890155004E6100E67
:10026000145C270E155806E20000DF2A010E01E398
:10027000DB2AEED700D0020EE15C02E2E16AE55231
:10028000E16EE552E7CFD9FF1200D9CFE6FFE1CF0B
:10029000D9FF020EE126DE6ADD6ADECF14F0DDCF83
:1002A00015F0D890155004E6C40E145C090E1558CC
:1002B00006E20000DF2A010E01E3DB2AEED700D0C0
:1002C000020EE15C02E2E16AE552E16EE552E7CF3F
:1002D000D9FF120000000000000000000000120022
:1002E000D9CFE6FFE1CFD9FF020EE126DE6ADD6A53
:1002F000DECF14F0DDCF15F0D890155004E6E80EEF
:10030000145C030E155806E20000DF2A010E01E31B
:10031000DB2AEED700D0020EE15C02E2E16AE55290
:10032000E16EE552E7CFD9FF1200D9CFE6FFE1CF6A
:10033000D9FF81940F0E8116FE0EDB504009F00BA1
:100340008112C8DFA6DE0F0E8116FE0EDB38F00B21
:10035000F00B8112BFDF9DDE00D0E552E7CFD9FF61
:10036000120000000000000000000000000000007B
:10037000000000000000000000000000000000007D
:10038000000000001200DACFE4FFE2CFDAFFE6520D
:100390009EA007D00101182B000E19231A231B233E
:1003A0009E90E552E5CFDAFF1100D9CFE6FFE1CF0D
:1003B000D9FF020EE126DE6ADD6AFD0EDBCFE9FF22
:1003C000FE0EDBCFEAFFEF5016E0FD0EDBCFE9FFBC
:1003D000FE0EDBCFEAFFEF50E66EE66A1FD8E5526D
:1003E000E552DF2A010E01E3DB2AFD0EDB2AFE0EB9
:1003F00001E3DB2AE2D7DECF14F0DDCF15F014C025
:10040000F3FF15C0F4FF020EE15C03E200D0E16AE5
:10041000E552E16EE552E7CFD9FF1200D9CFE6FFF2
:10042000E1CFD9FFACA2FED7FD0EDBCFE6FFE1ECBA
:100430000FF0E552E552E7CFD9FF1200D9CFE6FF22
:10044000E1CFD9FF020EE12601013C0E8E6F010EB5
:100450008F6F8EC1E6FF8FC1E6FFD950FB0FE96EAB
:10046000FF0EDA20EA6EEECFE6FFEECFE6FFEECF2C
:10047000E6FFEFCFE6FFFFEC0DF0146E060EE15E37
:1004800014508EC1E6FF8FC1E6FF8FDFE552E552C3
:10049000F3CFDEFFF4CFDDFF020EE15C02E2E16AA2
:1004A000E552E16EE552E7CFD9FF1200D9CFE6FF62
:1004B000E1CFD9FFD950FB0FE96EFF0EDA20EA6ECB
:1004C000D880000EEE54000EEE54000EEE54000ED6
:1004D000EE540CE2D950FB0FE96EFF0EDA20EA6E03
:1004E000EE06000EEE5AEE5AEE5AE4D7E552E7CF8A
:1004F000D9FF1200D9CFE6FFE1CFD9FF0E0EE126DA
:10050000F90EDBCFDEFFDBCFDDFFF80EDB5000089E
:1005100002E3070E08D0F80EDB50160802E2170EB1
:1005200002D0F80EDB28E66ED950080FE96EDACF5C
:10053000EAFFE552E750EE6EED6A020EDB6A030E4B
:10054000DB6AFB0EDBCF14F0FC0EDBCF15F0FD0EEB
:10055000DBCF16F0FE0EDBCF17F00A6A0B6A0C6ACF
:100560000D6A14C005F015C006F016C007F017C0DC
:1005700008F0CEEC0BF0010A33E1F90EDBCFE9FF16
:10058000DB2AFA0EDBCFEAFF01E3DB2A2D0EEF6E4A
:10059000FB0EDBCF14F0FC0EDBCF15F0FD0EDBCF36
:1005A00016F0FE0EDBCF17F00A6A0B6A800E0C6E97
:1005B000BF0E0D6E14C005F015C006F016C007F092
:1005C00017C008F029EC0BF0FB0E05C0DBFFFC0E9A
:1005D00006C0DBFFFD0E07C0DBFFFE0E08C0DBFF21
:1005E000FB0EDBCF14F0FC0EDBCF15F0FD0EDBCFE6
:1005F00016F0FE0EDBCF17F00A6A0B6A0C6A0D6A62
:1006000014C005F015C006F016C007F017C008F0BA
:10061000C5EC0BF0010A4AE1FB0EDBCF14F0FC0E37
:10062000DBCF15F0FD0EDBCF16F0FE0EDBCF17F0A3
:100630000A6A0B6A800E0C6E3F0E0D6E14C005F038
:1006400015C006F016C007F017C008F0CEEC0BF08E
:10065000010A2CE1146A156A200E166E410E176EFF
:10066000D950FB0FE96EFF0EDA20EA6EEECF05F0EF
:10067000EECF06F0EECF07F0EFCF08F014C00AF08F
:1006800015C00BF016C00CF017C00DF029EC0BF0E4
:1006900008C0EDFF07C0EDFF06C0EDFF05C0EFFF8E
:1006A000020EDB06030E01E2DB06B6D7FB0EDBCF44
:1006B00014F0FC0EDBCF15F0FD0EDBCF16F0FE0EB6
:1006C000DBCF17F00A6A0B6A200E0C6E410E0D6E1E
:1006D00014C005F015C006F016C007F017C008F0EA
:1006E000CEEC0BF0010A2EE0FB0EDBCF14F0FC0E7B
:1006F000DBCF15F0FD0EDBCF16F0FE0EDBCF17F0D3
:100700000A6A0B6A200E0C6E410E0D6E14C005F0C5
:1007100015C006F016C007F017C008F0D6EC0AF0B6
:10072000FB0E05C0DBFFFC0E06C0DBFFFD0E07C0A5
:10073000DBFFFE0E08C0DBFF020EDB2A030E01E327
:10074000DB2AB4D7020EDBCF14F0030EDBCF15F09B
:10075000D950080FE96EDACFEAFF1450EE26155093
:10076000ED22010EF36E040EF3CFDBFF050EDB6A04
:10077000040EDBCF06F0050EDBCF07F011EC0AF01C
:100780000A0E05C0DBFF0B0E06C0DBFF0C0E07C018
:10079000DBFF0D0E08C0DBFF040EDBCF14F0050EEF
:1007A000DBCF15F0080EDBCF16F0090EDBCF17F00C
:1007B00015501718E8AE02D0173404D01650145C48
:1007C000175015582EE20A0EDBCF14F00B0EDBCFBC
:1007D00015F00C0EDBCF16F00D0EDBCF17F00A6A0A
:1007E0000B6A200E0C6E410E0D6E14C005F015C084
:1007F00006F016C007F017C008F0D6EC0AF00A0E93
:1008000005C0DBFF0B0E06C0DBFF0C0E07C0DBFFD5
:100810000D0E08C0DBFF040EDB2A050E01E3DB2A08
:10082000BBD70A0EDBCF18F00B0EDBCF19F00C0E86
:10083000DBCF1AF00D0EDBCF1BF00A6A0B6A0C6AD5
:10084000400E0D6E18C005F019C006F01AC007F072
:100850001BC008F0D6EC0AF005C014F006C015F075
:1008600007C016F008C017F0D950FB0FE96EFF0E55
:10087000DA20EA6EEECF05F0EECF06F0EECF07F00D
:10088000EFCF08F014C00AF015C00BF016C00CF042
:1008900017C00DF040EC0AF008C0EDFF07C0EDFFF7
:1008A00006C0EDFF05C0EFFFFB0EDBCF14F0FC0E22
:1008B000DBCF15F0FD0EDBCF16F0FE0EDBCF17F011
:1008C0000A6A0B6A200E0C6E410E0D6E14C005F004
:1008D00015C006F016C007F017C008F0CEEC0BF0FC
:1008E000010A13E0FB0EDB6AFC0EDB6A800EF36E7E
:1008F000FD0EF3CFDBFF3F0EF36EFE0EF3CFDBFFFB
:10090000020EDB2A030E01E3DB2A020EDBCF14F01A
:10091000030EDBCF15F00001800E15145FE0F90E19
:10092000DBCFE9FFDB2AFA0EDBCFEAFF01E3DB2AAC
:10093000300EEF6EF90EDBCFE9FFDB2AFA0EDBCFCC
:10094000EAFF01E3DB2A2E0EEF6E080EDBCF14F078
:10095000090EDBCF15F0800E151414E0020EDBCF6C
:1009600016F0030EDBCF17F0080EDB50165C146E8A
:10097000090EDB501758156E020E14C0DBFF030E74
:1009800015C0DBFF040EDB68050EDB68040EDBCF51
:1009900014F0050EDBCF15F0020EDBCF16F0030EC0
:1009A000DBCF17F017501518E8AE02D0153404D07D
:1009B0001450165C1550175811E2F90EDBCFE9FF01
:1009C000DB2AFA0EDBCFEAFF01E3DB2A300EEF6E03
:1009D000040EDB06050E01E2DB06D8D7040EDB6A47
:1009E000050EDB6A040EDBCF14F0050EDBCF15F02D
:1009F000080EDBCF16F0090EDBCF17F015501718D5
:100A0000E8AE02D0173404D01650145C17501558B5
:100A100001E3ACD0FB0EDBCF05F0FC0EDBCF06F024
:100A2000FD0EDBCF07F0FE0EDBCF08F096EC0BF0EF
:100A3000060E06C0DBFF070E07C0DBFF300EE76EB9
:100A4000060EDBCF14F0070EDBCF15F0E7501426AF
:100A5000000E1522F90EDBCFE9FFDB2AFA0EDBCF01
:100A6000EAFF01E3DB2A14C0EFFF040EDBCF14F032
:100A7000050EDBCF15F0020EDB50141803E1030E58
:100A8000DB5015180BE1F90EDBCFE9FFDB2AFA0E7C
:100A9000DBCFEAFF01E3DB2A2E0EEF6E060EDBCF83
:100AA00006F0070EDBCF07F011EC0AF00A0E05C0C6
:100AB000DBFF0B0E06C0DBFF0C0E07C0DBFF0D0ECD
:100AC00008C0DBFF05C014F006C015F007C016F023
:100AD00008C017F0D950FB0FE96EFF0EDA20EA6E5E
:100AE000EECF05F0EECF06F0EECF07F0EFCF08F037
:100AF00014C00AF015C00BF016C00CF017C00DF0B2
:100B00003FEC0AF008C0EDFF07C0EDFF06C0EDFFA7
:100B100005C0EFFF146A156A200E166E410E176E9F
:100B2000D950FB0FE96EFF0EDA20EA6EEECF05F02A
:100B3000EECF06F0EECF07F0EFCF08F014C00AF0CA
:100B400015C00BF016C00CF017C00DF029EC0BF01F
:100B500008C0EDFF07C0EDFF06C0EDFF05C0EFFFC9
:100B6000040EDB2A050E01E3DB2A3CD7F90EDBCFAE
:100B7000E9FFFA0EDBCFEAFFEF6A0E0EE15C02E25C
:100B8000E16AE552E16EE552E7CFD9FF12000D0EA2
:100B9000E66EE66A43DCE552E5520A0EE66EE66A68
:100BA0003DDCE552E55212000F01030E386F070ECF
:100BB000926E92989296806A396B8168936AF19EE0
:100BC00061683A6B9468948094829484949C948E27
:100BD000D09C606A1200800E066E250E076E0650CD
:100BE00002E1C20E071824E0065002E1960E071833
:100BF0001AE0065002E14B0E071810E0800E0618AE
:100C000002E1250E071805E0820E0101006F016B5D
:100C100014D0820E0101006F016B0FD0400E010154
:100C2000006F016B0AD0200E0101006F016B05D02F
:100C30000A0E0101006F016B00D0400E006F016BC6
:100C400000C1E6FF01C1E6FF7C0EE66E0BEC0FF083
:100C5000E552E552E5529D989D9AF29CF29E120053
:100C60000F0149914993BD96BD84BD92BD80BF6A75
:100C7000BE6A9E949D941200D596D584D582D59057
:100C8000D59AD59C6A0EE66E670EE66EC5EC0FF03F
:100C9000E552E552F294F29AD59E12009480CD6A04
:100CA000CD82CD9ACD98CD96CD94CD8ECD9CCD9044
:100CB000CC6A1200100EE66E270EE66EE66AE66A51
:100CC00056EC02F0E552E552E552E5526DDF83DF66
:100CD0009EAA05D06BEC0FF00101046FF9D70C0E42
:100CE000E66EE66A0EEC02F0E552E552600EE66E44
:100CF000E30EE66E160EE66EE66A56EC02F0E5527C
:100D0000E552E552E55201010E6B0F6B050E0E5DCB
:100D1000000E0F5945E23C0E8C6F010E8D6F0EC117
:100D2000E9FF0FC1EAFF010ED890E936EA36E8067E
:100D3000FBE1600EE926000EEA22EECF14F0EFCFC1
:100D400015F0166A14C0E6FF15C0E6FF16C0E6FFF0
:100D50008CC1E6FF8DC1E6FF44EC0FF0176E050E67
:100D6000E15E17508CC1E6FF8DC1E6FFD5EC01F0C6
:100D7000E552E552F3CF12F1F4CF13F1F00EE66E27
:100D8000490EE66E020EE66EE66A56EC02F0E55299
:100D9000E552E552E55201010E2B000E0F23B6D7A6
:100DA0000EEC00F0010EE66E4EEC00F0E552880EFF
:100DB000E66E130EE66EE66AE66A56EC02F0E5525F
:100DC000E552E552E55201013C0E8C6F010E8D6F2C
:100DD0000E6B0F6B050E0E5D000E0F592DE2800E8F
:100DE000E66E4EEC00F0E5520EC1E9FF0FC1EAFFDE
:100DF000010ED890E936EA36E806FBE16E0EE926E8
:100E0000000EEA22EECFE6FFEFCFE6FF8AEC00F01D
:100E1000E552E552F00EE66E490EE66E020EE66E03
:100E2000E66A56EC02F0E552E552E552E552010160
:100E30000E2B000E0F23CED71FDF30DFBD6AF28CE2
:100E40009D90F29EF29C80A426D0010E01011C6FA1
:100E50001D6B6AC014F06BC015F0166A14C0E6FF73
:100E600015C0E6FF16C0E6FF8CC1E6FF8DC1E6FFA8
:100E700044EC0FF0176E050EE15E17508CC1E6FFD3
:100E80008DC1E6FFD5EC01F0E552E552F3CF12F14A
:100E9000F4CF13F125D0040E01011C6F1D6B6CC043
:100EA00014F06DC015F0166A14C0E6FF15C0E6FF19
:100EB00016C0E6FF8CC1E6FF8DC1E6FF44EC0FF0E3
:100EC000176E050EE15E17508CC1E6FF8DC1E6FF7F
:100ED000D5EC01F0E552E552F3CF12F1F4CF13F166
:100EE00056DE01010A6B0B6B00019F6B0101186B51
:100EF000196B1A6B1B6B1E6B1F6B226B236B206BAA
:100F0000216BCD906A0EE66E670EE66EC5EC0FF0B3
:100F1000E552E552000EE66EE66AA9EC0FF0E552E6
:100F2000E5529E9AF294D08E9E9080A405D0010E38
:100F300001011C6F1D6B04D0040E01011C6F1D6BA1
:100F4000F29CF28E0001826B836BF29AF2949D8088
:100F5000D58E8986CD80F2A4FED701010E6B0F6B72
:100F6000040E0E5D000E0F5904E20E2B000E0F232F
:100F7000F7D7010E00018225826F000E8321836F57
:100F8000F2946A0EE66E670EE66EC5EC0FF0E5525F
:100F9000E55201011C510001825D01011D5100015A
:100FA0008359D9E38996D59ECD908AEC0FF0F3CF83
:100FB0001EF1F4CF1FF1F294F29AF29E1EC106F0D8
:100FC0001FC107F00FEC0AF005C02EF106C02FF18B
:100FD00007C030F108C031F118C104F019C105F0A3
:100FE0001AC106F01BC107F024EC0AF005C014F08A
:100FF00006C015F007C016F008C017F00A6A0B6AA1
:10100000800E0C6E470E0D6E14C005F015C006F074
:1010100016C007F017C008F029EC0BF005C026F148
:1010200006C027F107C028F108C029F126C10AF03F
:1010300027C10BF028C10CF029C10DF02EC105F01D
:101040002FC106F030C107F031C108F040EC0AF0C2
:1010500005C02AF106C02BF107C02CF108C02DF104
:10106000800EE66E4EEC00F0E55201013C0E8C6FF6
:10107000010E8D6F80B436D00A6A0B6A800E0C6E3A
:10108000400E0D6E2AC105F02BC106F02CC107F0F1
:101090002DC108F0D6EC0AF005C02AF106C02BF1EC
:1010A00007C02CF108C02DF1010EE66E8CC1E6FFE1
:1010B0008DC1E6FF2AC1E6FF2BC1E6FF2CC1E6FF8A
:1010C0002DC1E6FF7AEC02F0146E070EE15E1450BB
:1010D000340EE66E6BEC00F0E552080E0101166F5F
:1010E000176B34D0310EE66E6BEC00F0E552010E5A
:1010F000E66E8CC1E6FF8DC1E6FF2AC1E6FF2BC17B
:10110000E6FF2CC1E6FF2DC1E6FF7AEC02F0146E7B
:10111000070EE15E14508CC1E6FF8DC1E6FF5DEC69
:101120000FF0E552E552F3CF12F1F4CF13F10101C4
:10113000020E125F000E135B3C0E1225E96E010ECB
:101140001321EA6EEF6A060E166F176B530EE66EEA
:101150006BEC00F0E552460EE66EE66A0EEC02F02D
:10116000E552E552720EE66EE66A0EEC02F0E552CA
:10117000E552650EE66EE66A0EEC02F0E552E552C7
:10118000710EE66EE66A0EEC02F0E552E5523D0E97
:10119000E66EE66A0EEC02F0E552E552200EE66ECF
:1011A000E66A0EEC02F0E552E5528CC1E6FF8DC115
:1011B000E6FF5DEC0FF0E552E552F3CF12F1F4CF0C
:1011C00013F10101146B156B106B116B1251165D4D
:1011D0001351175929E21251165D1351175919E28B
:1011E0003C0E1025E96E010E1121EA6EEF50E66EFD
:1011F0008D0E1425E96E000E1521EA6EE552E750BA
:10120000EF6E1207000E135B102B1123142B152306
:10121000E2D78D0E1425E96E000E1521EA6E2E0E12
:10122000EF6E142B000E1523030E165F000E175BD6
:101230001251165D1351175929E21251165D1351BF
:10124000175919E23C0E1025E96E010E1121EA6EC4
:10125000EF50E66E8D0E1425E96E000E1521EA6E34
:10126000E552E750EF6E1207000E135B102B1123AF
:10127000142B1523E2D78D0E1425E96E000E1521CF
:10128000EA6E2E0EEF6E142B000E1523030E165F62
:10129000000E175B1251165D135117591FE2000E15
:1012A000D8801255000E135519E23C0E1025E96E38
:1012B000010E1121EA6EEF50E66E8D0E1425E96ED7
:1012C000000E1521EA6EE552E750EF6E1207000E90
:1012D000135B102B1123142B1523E1D78D0E14252E
:1012E000E96E000E1521EA6E480EEF6E142B000E0B
:1012F00015238D0E1425E96E000E1521EA6E7A0E67
:10130000EF6E142B000E15238D0E1425E96E000EC2
:101310001521EA6EEF6A8D0EE66E000EE66E5DEC4C
:101320000FF0E552E552F3CF12F1F4CF13F10101C2
:101330000E0E125D000E13590AE2200EE66E6BECE3
:1013400000F0E5520101122B000E1323F0D78D0E91
:10135000E66E000EE66EADEC00F0E552E5528D0E45
:10136000E66E000EE66ED5EC01F0E552E552F3CFE5
:1013700012F1F4CF13F10BDC01010A2B000E0B2349
:10138000090ED8800A55000E0B5547E20A6B0B6B0D
:1013900080A422D06AC014F06BC015F0166A14C085
:1013A000E6FF15C0E6FF16C0E6FF8CC1E6FF8DC163
:1013B000E6FF44EC0FF0176E050EE15E17508CC18E
:1013C000E6FF8DC1E6FFD5EC01F0E552E552F3CF23
:1013D00012F1F4CF13F121D06CC014F06DC015F0F0
:1013E000166A14C0E6FF15C0E6FF16C0E6FF8CC102
:1013F000E6FF8DC1E6FF44EC0FF0176E050EE15ECF
:1014000017508CC1E6FF8DC1E6FFD5EC01F0E55227
:10141000E552F3CF12F1F4CF13F166D512000F9E0F
:1014200008D00F9E07AE05D0066C071EE86A07229B
:101430000F8E07C001F006C000F0136A126A8E0E0C
:10144000026E036A48EF0CF00F9E0CD00F9E07AEA1
:1014500009D0046C051E061E071EE86A0522062236
:1014600007220F8E07C001F006C000F005C013F080
:1014700004C012F09E0E026E036A48EF0CF00D7E5F
:101480000F6A84EC0CF09CEC0CF00FB62CEF0CF017
:101490000FA20AD00FAA03D00FBE2CEF0CF00FA49E
:1014A00038EF0CF035EF0CF00FAA05D00FAC38EF89
:1014B0000CF035EF0CF00FA00AD00FA808D00FBE2B
:1014C00004D00FA402D041EF0CF045EF0CF0126AEB
:1014D000036A0D50085C116E10E305C013F006C0DE
:1014E00000F007C001F008C010F00AC005F00BC002
:1014F00006F00CC007F00F3A09D00AC013F00BC079
:1015000000F00CC001F00DC010F0116C0F9E0FBC6C
:101510000F8E10C002F00FB074EF0CF01A0E1160B5
:1015200074EF0CF0026A086A0FA408D0056C061E5E
:10153000071E081EE86A0622072208220FAC08D000
:10154000136C001E011E021EE86A00220122022204
:10155000046A115207E008340732063205320432B9
:10156000112EF9D7055013260650002207500122EC
:101570000850022204C012F00F9E02AE0BD0126C73
:10158000131E001E011E021EE86A13220022012201
:1015900002220F8E02A006D0D88001320032133210
:1015A0001232102A10C002F048EF0CF00F6A84ECDF
:1015B0000CF09CEC0CF00FB62CEF0CF00FA205D049
:1015C0000FBA2CEF0CF033EF0CF00FBA3FEF0CF02A
:1015D0000FA005D00FB82CEF0CF03FEF0CF00FB8B8
:1015E00033EF0CF0036A7F0E0824026EE86A0322D0
:1015F0000D50025EE86A035A1A0E106E086A126AEB
:10160000136A006A016A0A50055E0B50065A0C50B4
:10161000075A000E085A09E70A5005260B50062201
:101620000C500722000E082201D0128AD8900536ED
:10163000063607360836D89012361336003601368D
:10164000102EE1D7075006100510D8A4128A48EFD3
:101650000CF00F6A84EC0CF09CEC0CF00FB62CEF45
:101660000CF00FA205D00FB82CEF0CF033EF0CF0FC
:101670000FAA05D00FB02CEF0CF033EF0CF00FB029
:1016800002D00FA802D03FEF0CF0036A0D500824DF
:10169000026EE86A03227E0E025EE86A035A126A4C
:1016A000136A006A016A0C500702F4CF01F0F3CF0D
:1016B00000F00B500702F3501326F4500022000EE6
:1016C00001220C500602F3501326F4500022000EA3
:1016D00001220A500702F3501226F4501322000E82
:1016E000002201220B500602F3501226F45013225E
:1016F000000E002201220C500502F3501226F45075
:101700001322000E002201220A500602F450122673
:10171000000E1322002201220B500502F450122663
:10172000000E13220022012248EF0CF00F6A84EC15
:101730000CF00FB6A0EF0BF00FA20ED00FB405D037
:101740007F0E076EFF0E066E1FD0800E076E066AB4
:101750001BD0076A066A18D00FB0FBD78F0E08603F
:10176000EDD77E0E0864F5D78E0E085C05E0D890A4
:1017700007320632082AF8D70FA406D0066C071ED7
:10178000E86A072207AEE5D71200D7EC0BF00FB6D8
:10179000000C0FB0000C0FB4000C010CD7EC0BF0D8
:1017A0000FB6000C0FB0000C0FA4000C010C0F6A58
:1017B00084EC0CF09CEC0CF00FB612000FAE08D0CD
:1017C0000FA004D00FA802D00F8012000F901200BB
:1017D0000D50085C0BE10C50075C08E10B50065CF7
:1017E00005E10A50055C02E10F801200D8A002D08A
:1017F0000F8E10D008500DC008F00D6E07500CC0B1
:1018000007F00C6E06500BC006F00B6E05500AC0B8
:1018100005F00A6E0D50085C10E0FF0F09E00F9014
:101820000FB403D00FAE0F8412000FAE0F9412004E
:101830000D2AD8900C320B320A320A50055E0B503A
:10184000065A0C50075A07BEEAD7D8900536063616
:101850000736082EF8D7C8D77F0E086EFF0E076E22
:10186000066E056E12007F0E0FBEFF0E086E02D0D0
:101870007F0E086E800E076E066A056AF3D70FAEFC
:1018800004D0800E086E076AF7D7086A076AF4D793
:101890000150001013101210F8E003BEF0D701BE83
:1018A0000CD002500310EBE0D890123613360036FD
:1018B00001360206D8A00306F2D70350D4E102286D
:1018C000D2E012AE11D07F0E121402E113A00CD0A0
:1018D000132AE86A0022012207E3D880013200328D
:1018E0001332022A0228BFE00250C9E013C005F0FB
:1018F00000C006F00134076E0230086E0732089E01
:101900000FBE088E32EF0CF00736083602E30F8464
:101910000F7E06E10F80086A076A066A056A1200F0
:10192000082803E0D88007321200D890073202E17D
:101930000F8212000F8612000C360D3602E30F8C58
:101940000F7E06E10F880D6A0C6A0B6A0A6A1200A4
:101950000D2803E0D8800C321200D8900C32EAE156
:101960000F8A1200008080808080800000C0C0C08C
:10197000C0C0C00000E0E0E0E0E0E00000F0F0F017
:10198000F0F0F00000F8F8F8F8F8F80000FCFCFCC3
:10199000FCFCFC0000FEFEFEFEFEFE0000FFFFFF62
:1019A000FFFFFF000010181C1E1C18100001030789
:1019B0000F070301040E1F0E0E0E0E0E0E0E0E0E5E
:1019C0000E1F0E0402040E111F100E0008040E114B
:1019D0001F100E0008040E010F110F000205020077
:1019E0000000000050726F6A6574206176656320A4
:1019F00050494331384632364B3232202B204C434B
:101A00004431783136202B204D6178333233322007
:101A10000D0A005061746820433A5C5F4331385CC2
:101A20005F4D657350726F6A6574735F4331385CE4
:101A3000467265715F506572696F640D0A00566584
:101A40007273696F6E3A2030352D31302D3230315E
:101A5000330D0A20506F727420636F6D6D20313921
:101A6000323030626473206F757665727420513D38
:101A700032304D687A0D0A00204672657175656EC8
:101A800063656D657472652031487A202E2E203191
:101A900030204D487A2C20436F72726563746966FA
:101AA0002031207365636F6E6465203D20340D0A1C
:101AB00020002054696D6572312053414E532070CF
:101AC00072657363616C6572203D20636F6D707425
:101AD000657572206427696D70756C73696F6E73BC
:101AE000200D0A002054696D657230203D20666526
:101AF0006E6574726520646520636F6D70746167D4
:101B000065202C62617365203120736563206176E6
:101B10006563205241323D31200D0A002054696D29
:101B2000657230203D2066656E657472652064655F
:101B300020636F6D7074616765202C62617365202E
:101B400034207365632061766563205241323D30F5
:101B5000200D0A0046726571656E63656D6574726D
:101B6000652020200031384632366B323220513D1C
:101B700032304D687A0067616D6D652031487A2E8C
:101B80002E31304D687A0031303025204D504C4197
:101B9000422043313820200076657273696F6E3AB7
:101BA00030352D31302D3133004D65737572206520
:101BB0006E2031206F752034730056696120657482
:101BC00061742064652052413220002020202020B2
:101BD0002020202020202020202020002020202025
:101BE000202020202020202020202020007061752F
:101BF0006C666A756A6F2E667265652E6600D9CF4F
:101C0000E6FFDACFE6FFF80EE3CFD9FFF90EE3CF18
:101C1000DAFFE652E652E652E652E652FB0EE124C5
:101C2000E76EFF0EE220E46EE652F30EE3CFE6FF2E
:101C3000F30EE3CFE6FFF30EE3CFE6FFF30EE3CFC1
:101C4000E6FF84EC0EF0F50EE124E96EFF0EE220D3
:101C5000EA6E71EC0EF019E174EC0EF018E171EC23
:101C60000EF017E174EC0EF016E171EC0EF015E1D8
:101C700074EC0EF014E171EC0EF013E174EC0EF064
:101C800012E171EC0EF011E112D07AEC0EF07FEC63
:101C90000EF07AEC0EF07FEC0EF07AEC0EF07FECAA
:101CA0000EF07AEC0EF07FEC0EF07AEC0EF07FEC9A
:101CB0000EF0DE6AF50EE126FF0EE222FF0EE3CF04
:101CC000DAFFE552FF0EE3CFD9FFE552FA0EE12429
:101CD000E96EFF0EE220EA6EEECFF3FFEFCFF4FFE6
:101CE0001200EF380F0B1200EF500F0B02E1EE5213
:101CF000D8841200EF380F0B300FDE6E1200EE505A
:101D00000F0B300FDE6E1200FA0EE3CFE9FFFB0E71
:101D1000E3CFEAFF200EE66EEE6AEE6AEE6AEE6A46
:101D2000EF6AD890FB0EE336FC0EE336FD0EE33689
:101D3000FE0EE336ED36ED36ED36ED36EF36FF0EC0
:101D4000E3060FE0B3EC0EF0EE52B3EC0EF0EE5201
:101D5000B3EC0EF0EE52B3EC0EF0EE52B3EC0EF02C
:101D6000E1D7E56E1200030EEF24E8B6EF6E300EF9
:101D7000EF24E8BEEF6E000C0E0EF66E000EF76E4E
:101D8000000EF86E01010900F550F86F0900F550DA
:101D9000F96F03E1F86701D03DD00900F550F36F0A
:101DA0000900F550F46F0900F550F56F09000900BE
:101DB000F550E96E0900F550EA6E090009000900C6
:101DC000F550F66F0900F550F76F09000900F6CFDE
:101DD000FAF1F7CFFBF1F8CFFCF1F3C1F6FFF4C154
:101DE000F7FFF5C1F8FF0101F65302E1F75307E0F1
:101DF0000900F550EE6EF607F8E2F707F9D7FAC1D9
:101E0000F6FFFBC1F7FFFCC1F8FF0101F807000E68
:101E1000F95BBFD71200D9CFE6FFDACFE6FFE1CFFB
:101E2000D9FFE2CFDAFFAC6AAB6AFD0EDBB0AC885B
:101E3000DBA202D0AC8CAB8CDBB4AC8EDBA602D0C8
:101E4000AB8801D0AB8ADBB8AC84DBBAAB86DBAC49
:101E500002D09D8A01D09D9ADBAE02D09D8801D030
:101E60009D98FB0EDB50AF6EFC0EDBCF15F015C05E
:101E700014F0156A1450B06EAC8AAB8EE552E5CF03
:101E8000DAFFE7CFD9FF1200FB0EE3CFF6FFFC0E1F
:101E9000E3CFF7FFFD0EE3CFF8FFFE0EE3CFE9FF40
:101EA000FF0EE3CFEAFFE9CFF3FFEACFF4FF09002B
:101EB000F5CFEFFFEE66FBD71200FE0EE3CFE9FF92
:101EC000FF0EE3CFEAFFF36AF46AEE5203E0F34A4F
:101ED000F42AFBD71200D9CFE6FFDACFE6FFE1CF35
:101EE000D9FFE2CFDAFFE652F20E0101FD17ABACEB
:101EF00003D0FD91ABB0FD81ABB4FD85ABB2FD87E6
:101F0000AE50DF6EDF50E552E552E5CFDAFFE7CFA6
:101F1000D9FF1200D9CFE6FFDACFE6FFE1CFD9FF34
:101F2000E2CFDAFFE652E652CE50DF6E010ECFCF9F
:101F3000DBFFDECF14F0DDCF15F014C0F3FF15C0CA
:101F4000F4FFE552E552E552E5CFDAFFE7CFD9FFDE
:101F50001200D9CFE6FFDACFE6FFE1CFD9FFE2CF1B
:101F6000DAFFE652E652FC0EDBCFDEFFDBCFDDFF11
:101F7000010EDB50CF6EDF50CE6EE552E552E552DA
:101F8000E5CFDAFFE7CFD9FF1200D9CFE6FFDACFEE
:101F9000E6FFE1CFD9FFE2CFDAFFE652E652FC0ED0
:101FA000DBCFDEFFDBCFDDFF010EDB50D76EDF5076
:101FB000D66EE552E552E552E5CFDAFFE7CFD9FF1D
:101FC0001200D9CFE6FFDACFE6FFE1CFD9FFE2CFAB
:101FD000DAFFACAC04D0AC900101FDB3AC80FD0ED7
:101FE000DB50AD6EE552E5CFDAFFE7CFD9FF120047
:101FF000380EF36E00EE00F00F0E01D81200EA600A
:1020000002D0EE6AFCD7F350E9601200EE6AFCD70A
:102010001EEE00F02EEE00F0F86A0F9CBCEC0EF005
:1020200003EC00F05AEC06F0FBD71200E419131A87
:102030003E1A781AB21AE41A1C1B541B651B761B35
:10204000871B981BA91BBA1BCB1BDC1BED1B0000BD
:102050003030303030303030003132333435363794
:10206000383930313233343536370000FFFFFFFF67
:10207000FFFFFFFFFFFFFFFFFFFFFFFFFFFFFFFF70
:10208000FFFFFFFFFFFFFFFFFFFFFFFFFFFFFFFF60
:10209000FFFFFFFFFFFFFFFFFFFFFFFFFFFFFFFF50
:1020A000FFFFFFFFFFFFFFFFFFFFFFFFFFFFFFFF40
:0200000400F00A
:020000040030CA
:0E0000000022193C009D84000FC00FE00F404D
:020000040020DA
:08000000FFFFFFFFFFFFFFFF00
:00000001FF
